:100000000C947A020C94BE020C94BE020C94BE02B4
:100010000C94BE020C94BE020C94BE020C94BE0260
:100020000C94BE020C94BE020C94620D0C94340E1F
:100030000C94BE020C94BE020C94BE020C94BE0240
:100040000C94BE020C943E220C94BE020C94BE0290
:100050000C94BE020C94D11B0C94BE020C94BE02F4
:100060000C94BE020C94BE020C94BE020C94BE0210
:100070000C94BE020C94BE020C94BE020C94BE0200
:100080000C94BE020C94BE020C94BE020C94BE02F0
:100090000C94BE020C94BE020C94BE020C94BE02E0
:1000A0000C94BE020C94BE020C94BE02A10EC30EB0
:1000B000B10FC30EB10F080F2B0FB10F800F930FAD
:1000C0006212621291129112C712E71218141814D8
:1000D000F2121814A213A2130914181418141214EB
:1000E000AF13AF13AF13AF13AF13AF13AF13AF1300
:1000F000AF13AF13AF13AF13AF13AF13AF13AF13F0
:10010000C113CE13D513DC13E6130000F0A12E00AB
:100110004C002A00E100354100001E0014000400DC
:100120001D7134004D001F001A0015001B00E10472
:100130002A00200009001600060050002C002100B3
:100140001300170019004F004A0022000A000700A0
:10015000050000006574500001540000007F00009D
:10016000E3004F000154000000770000E20023008C
:100170000D000B000E000000297124000F0011007B
:10018000100052004B0025001800080036005100F6
:10019000280026001C000C0037002F002B00270031
:1001A00033001242387130004E002D00310034000F
:1001B000E500C10000000100010001000100010094
:1001C00000003A001E0220022202010001003B0052
:1001D0001F0221022302010001003C002F0226021F
:1001E0002F00010001003D00300227023000010015
:1001F00001003E003102350035020000010001001F
:1002000001000000010000000100010001000000E9
:100210000100000001003F005200510024020000D4
:1002200001004000240021001E00010001004100E7
:10023000250022001F003700010042002600230095
:10024000200027000100430025022E0231002E006D
:100250000100440045000100010001000000010010
:100260000100010001000100000001000100010087
:1002700001000100010001000100F2000100010085
:1002800001000100F000F1000100F4000100010094
:100290000100F3000100F500010001000100010070
:1002A0000100000001000100010000000100000049
:1002B0000100010001000000010000000100010038
:1002C0000100010001000000010001000100010027
:1002D0000100A9000100010001000100AC00AA001A
:1002E000B600010001000100AB00A8000100010000
:1002F0000100010001000100010001000100AE0049
:1003000001000100000016034500720067006F0045
:1003100044006F007800200045005A0000001603DA
:100320004500720067006F0044006F0078002000F5
:1003300045005A0000000403090409026D0004018D
:1003400000A0FA09040000010301010009211101C4
:100350000001223F000705810308000A090401008B
:100360000103010200092111010001224D000705CE
:10037000820308000A0904020001030000000921A9
:10038000110100012236000705830308000A090451
:1003900003000103000000092111010001223900BE
:1003A000070584031000011201100100000008ED90
:1003B000FE071301000102000105010906A1010564
:1003C0000719E029E7150025019508750181020547
:1003D000081901290595057501910295017503918B
:1003E0000105071900297715002501957875018108
:1003F00002C005010980A101850216010026B7008F
:100400001A01002AB700751095018100C0050C097A
:1004100001A1018503160100269C021A01002A9CF5
:1004200002751095018100C005010902A1010901B1
:10043000A10005091901290515002501950575017A
:10044000810295017503810105010930093115818A
:10045000257F95027508810609381581257F95014C
:1004600075088106050C0A38021581257F950175EE
:10047000088106C0C005010906A101050719E02988
:10048000E715002501950875018102950175088120
:100490000105081901290595057501910295017558
:1004A0000391010507190029FF150025FF95067521
:1004B000088100C0000000000000000000000001F2
:1004C0000204060A0F17202C3A4A5D71879DB3C7B4
:1004D000DAE9F5FCFFFCF5E9DAC7B39D87715D4AFF
:1004E0003A2C20170F0A0604020100000000000049
:1004F0000000000011241FBECFEFDAE0DEBFCDBF49
:1005000004B603FE24C08091FB019091FC01A091F0
:10051000FD01B091FE018730904BA740B04BB9F47C
:100520001092FB011092FC011092FD011092FE014D
:1005300014BE84B7877F84BF88E10FB6F894809398
:100540006000109260000FBEE0E0FFE3099511E04B
:10055000A0E0B1E0EAE0F8E402C005900D92A43317
:10056000B107D9F711E0A4E3B1E001C01D92AB3FA0
:10057000B107E1F70E94A60A0C9403240C94000032
:100580001092B9008AE08093B800089594EA90939D
:10059000BC009091BC0097FFFCCF9091B900987F70
:1005A000983021F0903111F081E008958093BB00E4
:1005B00084E88093BC008091BC0087FFFCCF8091D1
:1005C000B900887F883111F0803471F780E0089598
:1005D00084E98093BC008091BC0084FDFCCF089529
:1005E0008093BB0084E88093BC008091BC0087FFAF
:1005F000FCCF9091B900987F81E0983209F480E0B7
:10060000089584E88093BC008091BC0087FFFCCFF4
:100610008091BB00089580910101811115C080E493
:100620000E94C6028093010181110CC082E10E94E8
:10063000F00280930101811105C08FEF0E94F0024A
:10064000809301010E94E80284B1807F84B985B162
:10065000807F85B98AB1837F8AB98BB1837F8BB95B
:100660003E98469808950E94C604809301010E9416
:100670000B0380B38C7080BB81B3836F81BBA5E318
:10068000B1E0E3E4F1E08EE08E0F11921D928E1343
:10069000FCCF0C94B004BF92CF92DF92EF92FF9206
:1006A0000F931F93CF93DF9380910101882379F0FB
:1006B000809134018F5F80933401811108C00E94C2
:1006C000C60480930101811102C00E94580405E311
:1006D00011E0C0E0D0E0DD24D39482E0C82EEE2407
:1006E000E394F12CC730D10500F58091010181110F
:1006F00064C080E40E94C60280930101811112C08F
:1007000082E10E94F0028093010181110BC0C701B8
:100710000C2E01C0880F0A94EAF780950E94F0021F
:10072000809301010E94E80248C0CA30A1F028F479
:10073000C83059F0C93061F005C0CC3089F070F094
:10074000CD3089F0209A289810C0219A29980DC0A0
:10075000229A2A980AC0239A2B9807C0529A01C05D
:10076000539A5B9802C03E9A469890EA9A95F1F7A0
:100770009FB1799902C082E001C080E091709D250F
:10078000982B7C9902C084E001C080E0892B7D9980
:1007900002C038E001C030E0832B7E9902C020E126
:1007A00001C020E0822B9FB19095991F9927991F36
:1007B0009295990F907E892B0FC080910101811134
:1007C00049C080E40E94C60280930101882379F128
:1007D000B12C0E94E8028B2DF8019081981719F036
:1007E0008083C09200010E940B0321960F5F1F4F70
:1007F000CE30D10509F076CF80910001882361F1D8
:10080000815080930001882339F08FE99FE00197A0
:10081000F1F700C0000020C0A3E4B1E0E5E3F1E09F
:10082000CF01825F91919D938E13FCCF15C083E120
:100830000E94F002809301018111CACF81E40E94DD
:10084000C602809301018111C3CF0E940103B82E1B
:10085000B094BFCF80E0C0CF0E94560481E0DF910A
:10086000CF911F910F91FF90EF90DF90CF90BF90AD
:100870000895E82FF0E0ED5BFE4F80810895089524
:100880000F931F93CF93DF93C3E4D1E010E00C2FBD
:10089000025F899190E00E94F71A180F0C13F9CFAC
:1008A000812FDF91CF911F910F9108950C94260510
:1008B00056985E9825982D9826982E9827982F98C8
:1008C0008FEF90E0909389008093880090938B0045
:1008D00080938A0090938D0080938C00259A2D9AA6
:1008E0002FEF80E792E0215080409040E1F700C078
:1008F0000000269A2E9A2FEF80E792E02150804048
:100900009040E1F700C00000279A2F9A2FEF80E770
:1009100092E0215080409040E1F700C0000025980F
:100920002D982FEF80E792E0215080409040E1F732
:1009300000C0000026982E982FEF80E792E021500B
:1009400080409040E1F700C0000027982F9856980B
:100950005E9825982D9826982E9827982F98089578
:1009600089EA8093800089E08093810024982C9804
:100970003F988AB18F748AB96E98479A8BB1806B11
:100980008BB9769A0E9458040C94250580E28093D6
:1009900001018091510181110EC00E94C00281E0CD
:1009A000809351012FEF83ED90E3215080409040E0
:1009B000E1F700C0000080E40E94C60280930101BC
:1009C00081112EC00E94F00280930101811128C084
:1009D0000E94F00280930101811122C08FE30E94E6
:1009E000F0028093010181111BC00E94E80280E4A3
:1009F0000E94C60280930101811112C08CE00E9406
:100A0000F0028093010181110BC00E94F0028093DB
:100A10000101811105C08FE30E94F0028093010162
:100A20000E94E80280910101089561110BC0FC0150
:100A30008281882321F085EE0E94061103C085EE95
:100A40000E94CE1180E090E0089508956091BD016C
:100A50007091BE018091BF019091C0010E94031B63
:100A600056985E9825982D9826982E9827982F9816
:100A7000813019F0823021F00895259A2D9A089539
:100A8000269A2E9A089581E0089581E008950C94A5
:100A9000450508950F931F93CF93DF938C01FC01BD
:100AA000C081D181CE010E947C19BE010E94F30554
:100AB000EC01B8010E944705882309F48DC0F801B4
:100AC0008281882309F44AC080915D0181111FC091
:100AD000C431F0E5DF0709F051C00E94490581E00B
:100AE00080935D010E949B1B90935C0180935B014E
:100AF0001092540110925601109255011092580113
:100B00001092570110925A011092590165C08091BC
:100B10005B0190915C010E94A71B883C910570F4D9
:100B200080915401E82FF0E0EE0FFF1FEB5AFE4FCB
:100B3000D183C0838F5F809354014EC0C43880E559
:100B4000D80721F0C538D04501F13AC0F8018281BB
:100B5000882341F01092520182E01EC0C438E0E5C3
:100B6000DE0759F580915201811106C086E20E948C
:100B7000061186E20E94CE1182E01CC0C438F0E566
:100B8000DF0741F3C538D045D9F4F80182818823C5
:100B900031F01092530180E20E941D121DC080911D
:100BA0005301811106C087E20E94061187E20E946C
:100BB000CE1180E20E9424120FC0C538D04529F31F
:100BC00081E08093520180935301C801DF91CF915E
:100BD0001F910F910C94430580E0DF91CF911F91FD
:100BE0000F910895089596E0799FF001112494E5FE
:100BF000899FE00DF11D1124E60FF11DEE0FFF1F7F
:100C0000E25FFE4F859194910895880F991FFC0132
:100C1000E657F040859194910895880F991FFC0143
:100C2000E65FFE4F8591949108950F931F93CF93A4
:100C3000DF93EC01811520E3920750F5C11580E2A6
:100C4000D80708F0C3C0CB3BD10590F4C83AD10512
:100C500008F06AC0C53AD10508F05BC0C430D105C0
:100C600008F0D0C1219709F0CAC101E010E00AC222
:100C7000CF3FD10511F008F0C5C1C03FD10508F044
:100C8000A2C0CE01805E9109089708F4BBC1B7C12C
:100C9000C13090E5D90709F4A2C020F5C0318FE436
:100CA000D80770F4C11590E4D90708F094C0C115B5
:100CB00021E3D20708F0A3C1DD278E01106CE2C149
:100CC000C115D04509F09BC10E9483148FEF94E3B6
:100CD0002CE0815090402040E1F700C000000E94CD
:100CE000F61BD0C1C11597E5D90758F4C03121E5ED
:100CF000D20708F01CC1C43180E5D80708F475C0DC
:100D00007EC1CE0190578115904108F078C1DF7007
:100D100073C1C53AD10509F477C1C63AD10509F0C6
:100D200076C102E810E4AEC1C83AD10509F472C137
:100D3000C93AD10509F471C1CA3AD10509F470C1A3
:100D4000CB3AD10509F46FC1CC3AD10509F46EC193
:100D5000CD3AD10509F46DC1C03BD10509F46CC190
:100D6000CE3AD10509F46BC1CF3AD10509F46AC175
:100D7000C13BD10509F469C1C23BD10509F468C181
:100D8000C33BD10509F467C1C43BD10509F466C171
:100D9000C53BD10509F465C1C63BD10509F464C161
:100DA000C73BD10509F463C1C83BD10509F462C151
:100DB000C93BD10509F461C1CA3BD10509F460C141
:100DC00000E014E45FC18E0110655CC1CE019F702C
:100DD0000E940D0658C1DF708E01106A53C18091C8
:100DE000DA0181608093DA014DC10E949B1D81115F
:100DF00002C00E94811D0E94B81D90E09093FB01EB
:100E00008093FA01C23080E5D80721F48091FA017D
:100E1000816086C0C43090E5D90721F48091FA0141
:100E200082607EC0C63020E5D20721F48091FA01AD
:100E3000846076C0C83080E5D80719F48091FA0143
:100E400027C0CA3090E5D90721F48091FA0180616A
:100E500067C0CC3020E5D20721F48091FA0180628E
:100E60005FC0CE3080E5D80721F48091FA0180641C
:100E700057C0C03190E5D90721F48091FA0180680C
:100E80004FC0C23120E5D20729F48091FA01846075
:100E9000886046C0C33080E5D80721F48091FA010C
:100EA0008E7F3EC0C53090E5D90721F48091FA01CC
:100EB0008D7F36C0C73020E5D20721F48091FA013A
:100EC0008B7F2EC0C93080E5D80719F48091FA01D4
:100ED00026C0CB3090E5D90721F48091FA018F7EAE
:100EE0001FC0CD3020E5D20721F48091FA018F7D1B
:100EF00017C0CF3080E5D80721F48091FA018F7BAD
:100F00000FC0C13190E5D90721F48091FA018F77A4
:100F100007C0C331D04531F48091FA018B7F877FC0
:100F20008093FA018091FA010E94BC1DABC08D2F05
:100F300099278F70992781309105D9F49E012370EC
:100F4000332702C0880F991F2A95E2F79C688E010B
:100F500044E0000F111F4A95E1F700271370802B22
:100F6000912B53E0CC0FDD1F5A95E1F7C076DD27BA
:100F70002FC08230910531F4DC2FCC278E01016F18
:100F8000106A80C08330910569F4CE01837099277F
:100F900001E010E002C0000F111F8A95E2F7C801BE
:100FA0009C680FC084309105B9F4CE0183709927F5
:100FB00001E010E002C0000F111F8A95E2F7C8019E
:100FC0009A6823E0CC0FDD1F2A95E1F7C07ED77029
:100FD0008C010C2B1D2B56C08530910531F4DC2F74
:100FE000CC278E01046F106A4DC0069709F04AC0E5
:100FF000CF71DD27DC2FCC278E01106243C000E0CB
:1010000010E040C08E013EC001E810E43BC003E8A0
:1010100010E438C002EE14E435C009EE14E432C026
:101020000AEE14E42FC005EB14E42CC006EB14E424
:1010300029C007EB14E426C00CEC14E423C00DEC2B
:1010400014E420C003E815E41DC00AE815E41AC042
:1010500002E915E417C004E915E414C001E216E43E
:1010600011C003E216E40EC004E216E40BC005E270
:1010700016E408C006E216E405C007E216E402C062
:101080000AE216E4C801DF91CF911F910F910895F4
:1010900096E0799FF001112494E5899FE00DF11D00
:1010A0001124E60FF11DEE0FFF1FE25FFE4F859149
:1010B0009491803E9105E0F4803C910558F5813390
:1010C000910509F46FC048F48932910509F463C0B1
:1010D0008A32910509F46DC072C089339105E9F037
:1010E00082389105D1F08533910509F44DC067C070
:1010F000833E910581F138F4803E9105B9F0823E3E
:101100009105D9F05CC0863E910561F1873E91055D
:10111000A1F155C00E94050608952091FA0120FD15
:1011200002C021FF4CC080EE90E049C08091FA01DE
:1011300080FFF9CF89E390E042C08091FA0182FFFD
:101140000EC08091FA0184FF03C080E090E037C0B8
:1011500083EE90E034C08091FA0182FFF2CF82EEFC
:1011600090E02DC08091FA0183FF0BC08091FA01BD
:1011700084FDEBCF87EE90E022C08091FA0183FFDF
:10118000F5CF86EE90E01BC08091FA0185FF07C085
:1011900089E290E014C08091FA0185FFF9CF85E3E0
:1011A00090E00DC08091FA0186FF07C08AE290E0CE
:1011B00006C08091FA0186FFF9CF81E390E00E949A
:1011C0001506089508950C94E20880916E01089523
:1011D000CF93DF9300D01F92CDB7DEB79C018091F3
:1011E000F101843019F593E099833B832A8390932E
:1011F000E9008FEF9091E800815095FD06C095EDD4
:101200009A95F1F700008111F5CF8091E80085FFF4
:101210000DC040E050E063E070E0CE0101960E9416
:10122000520B8091E8008E778093E8000F900F902A
:101230000F90DF91CF910895CF93DF9300D01F924D
:10124000CDB7DEB72091F101243021F522E02983CA
:101250009B838A8383E08093E9008FEF9091E8007D
:10126000815095FD06C095ED9A95F1F7000081112A
:10127000F5CF8091E80085FF0DC040E050E063E0CD
:1012800070E0CE0101960E94520B8091E8008E77AB
:101290008093E8000F900F900F90DF91CF91089509
:1012A0002091F1012430F1F422E02093E9002FEFA6
:1012B0003091E800215035FD06C035ED3A95F1F743
:1012C00000002111F5CF2091E80025FF0BC040E080
:1012D00050E065E070E00E94520B8091E8008E774C
:1012E0008093E8000895CF93DF93EC019091F10192
:1012F000943009F046C080910C018823D9F0809188
:101300000D018823B9F09093E9008FEF9091E800E8
:10131000815095FD06C095E19A95F1F70000811185
:10132000F5CF8091E80085FF2CC040E050E060E1FF
:1013300070E017C081E08093E9008FEF9091E800A2
:10134000815095FD06C095ED9A95F1F70000811149
:10135000F5CF8091E80085FF14C040E050E068E0E0
:1013600070E0CE010E94520B8091E8008E7780934E
:10137000E80080E1FE01AEE5B1E001900D928A95B2
:10138000E1F7DF91CF9108958091F001811109C0BB
:101390000E94E70C0E94440D8091E20084608093DB
:1013A000E20008951092F001089508950C942B2204
:1013B0000E948C1B0E9431220E94EA0F0C94E308C9
:1013C00042E061EC81E00E94610C42E061EC82E06D
:1013D0000E94610C42E061EC83E00E94610C42E1FA
:1013E00061EC84E00C94610C8091F301833009F48A
:1013F00055C030F4813071F0823009F48EC0089508
:101400008A3009F47AC08B3009F460C0893009F061
:101410009CC020C08091F201813A09F096C0809171
:10142000E800877F8093E8008091F6019091F701B2
:10143000892B21F460E18EE591E003C060E080E05B
:1014400090E070E00E949D0B8091E8008B77809384
:10145000E80008958091F201813209F076C0809110
:10146000F6019091F701009719F0039709F06DC00C
:101470008091E800877F8093E8008091E80082FDFA
:1014800005C08091F1018111F8CF5FC08091F1001A
:1014900080936E018091E8008B7753C08091F201B8
:1014A000813A09F052C08091F6019091F701892BA1
:1014B00009F04BC08091E800877F8093E80080911D
:1014C000E80080FFFCCF80910C0136C08091F201D2
:1014D0008132D9F58091F6019091F701892BA9F518
:1014E0008091E800877F8093E8000E94960C8091AD
:1014F000F40180930C010C9483148091F2018132E9
:1015000021F58091E800877F8093E8000E94960C87
:101510008091F50180936F0108958091F201813AE5
:10152000A1F48091E800877F8093E8008091E80033
:1015300080FFFCCF80916F018093F1008091E800E3
:101540008E778093E8000C94960C089584B7877F7B
:1015500084BF88E10FB6F894809360001092600019
:101560000FBE90E080E80FB6F894809361009093EE
:1015700061000FBE0E9439100E94E70C0E94440DCA
:101580008091E20084608093E20078940E94CA0F08
:101590000E943B1082E091E00E94E50F0E94192218
:1015A0008091F101853069F40E94531B8091EF0115
:1015B0008823B1F30E947E1B882391F30E943C0B89
:1015C000EFCF0E944110ECCF292F33272330310574
:1015D000C9F064F42130310581F02230310509F081
:1015E00043C08DE690E02AE333E042C0213231056A
:1015F000F1F02232310541F137C082E190E027EA73
:1016000033E036C099278130910541F08230910551
:1016100041F0892B49F5E6E3F3E005C0EEE1F3E0A4
:1016200002C0E6E0F3E0849190E09F0121C06430C5
:10163000D8F4E62FF0E0EE0FFF1FEE5DFE4F2081A5
:10164000318189E090E014C0643070F470E0FB01F7
:10165000EE0FFF1FE65EFE4F20813181FB01EA5E47
:10166000FE4F808190E004C080E090E020E030E018
:10167000FA0131832083089580E189BD82E189BD2B
:1016800009B400FEFDCF8091D8008F7D8093D800F3
:101690008091E00082608093E0008091E00081FD15
:1016A000FCCF0895CF92DF92EF92FF920F931F939A
:1016B000CF93DF93EC018B016A010E94B50C81117D
:1016C00033C0C114D10439F0F60180819181081B27
:1016D000190BC80FD91FE12CF12C0115110519F1B7
:1016E0008091E80085FD16C08091E8008E77809398
:1016F000E800C114D10449F0F60180819181E80E1F
:10170000F91EF182E08285E00FC00E94B50C8823AB
:1017100021F30AC089918093F10001501109FFEF74
:10172000EF1AFF0ADACF80E0DF91CF911F910F917E
:10173000FF90EF90DF90CF9008952091F8013091C5
:10174000F9012617370748F06115710539F4209122
:10175000E8002E772093E80001C0B90140E0611550
:101760007105A9F12091F101222309F443C025302C
:1017700009F442C02091E80023FD40C02091E80018
:1017800022FD32C02091E80020FFE9CF4091F30014
:101790002091F20030E0342BFC01CF01611571057E
:1017A00059F02830310540F481918093F100615067
:1017B00071092F5F3F4FF1CF41E02830310509F02B
:1017C00040E02091E8002E772093E800C8CF411137
:1017D000C9CF0AC08091F101882361F0853061F0A2
:1017E0008091E80083FD0AC08091E80082FFF2CF7B
:1017F00080E0089582E0089583E0089581E00895EF
:101800002091F8013091F9012617370748F061154A
:10181000710539F42091E8002E772093E80001C08B
:10182000B901FC0120E06115710591F18091F10190
:10183000882309F440C0853009F43FC08091E80056
:1018400083FD3DC08091E80082FD2FC08091E800BB
:1018500080FFE9CF2091F3008091F20090E0922B7D
:101860006115710559F08830910540F42491209359
:10187000F1003196615071090196F2CF21E008978D
:1018800009F020E08091E8008E778093E800CBCFCC
:101890002111CCCF0AC08091F101882361F08530FD
:1018A00061F08091E80083FD0AC08091E80082FF2A
:1018B000F2CF80E0089582E0089583E0089581E00A
:1018C0000895982F973058F59093E900981739F0BC
:1018D0007091EC002091ED005091F00003C0242F96
:1018E000762F50E021FF19C03091EB003E7F3093FE
:1018F000EB003091ED003D7F3093ED003091EB0037
:1019000031603093EB007093EC002093ED00509326
:10191000F0002091EE0027FF07C09F5FD3CF8F70AC
:101920008093E90081E0089580E008958091F201BC
:1019300087FF11C08091E80082FD05C08091F10110
:101940008111F8CF11C08091E8008B770BC0809196
:10195000F101882349F08091E80080FFF8CF809161
:10196000E8008E778093E80008952091E40030919C
:10197000E50095E64091EC00842F817040FF22C085
:101980008091E80080FD1CC08091F101882391F0D6
:10199000853091F08091EB0085FD10C04091E4000E
:1019A0005091E5004217530729F39A01915011F71E
:1019B00084E0089582E0089583E0089581E0089529
:1019C00080E008954091E80042FFDECF08950E9434
:1019D000550D0E945D0DE0EEF0E080818160808316
:1019E000E8EDF0E080818F77808319BCA7EDB0E04F
:1019F0008C918E7F8C9380818F7E80831092F001FA
:101A000008950F931F93CF93DF930E94550D0E946B
:101A10005D0DC8EDD0E088818F77888388818068EC
:101A2000888388818F7D888319BC1092F101109280
:101A3000ED011092EF011092EE0100EE10E0F801BE
:101A400080818B7F808388818160888342E060E031
:101A500080E00E94610CE1EEF0E080818E7F808367
:101A6000E2EEF0E080818160808380818860808305
:101A7000F80180818E7F8083888180618883DF91F7
:101A8000CF911F910F910895E8EDF0E080818F7E56
:101A90008083E7EDF0E080818160808384E082BF15
:101AA00081E08093F0010C94010DE8EDF0E080817D
:101AB0008E7F80831092E20008951092DA001092D7
:101AC000E10008951F920F920FB60F9211242F93E9
:101AD0003F934F935F936F937F938F939F93AF93B6
:101AE000BF93EF93FF938091E10082FF0BC0809141
:101AF000E20082FF07C08091E1008B7F8093E100CC
:101B00000E94C90F8091DA0080FF1FC08091D80029
:101B100080FF1BC08091DA008E7F8093DA00809175
:101B2000D90080FF0DC080E189BD82E189BD09B483
:101B300000FEFDCF81E08093F1010E94C40905C041
:101B400019BC1092F1010E94D2098091E10080FF3E
:101B500019C08091E20080FF15C08091E2008E7F65
:101B60008093E2008091E20080618093E2008091A6
:101B7000D80080628093D80019BC85E08093F10181
:101B80000E94D6098091E10084FF30C08091E2007C
:101B900084FF2CC080E189BD82E189BD09B400FECB
:101BA000FDCF8091D8008F7D8093D8008091E10097
:101BB0008F7E8093E1008091E2008F7E8093E2002F
:101BC0008091E20081608093E2008091ED018823A2
:101BD00011F084E007C08091E30087FD02C081E03E
:101BE00001C083E08093F1010E94D8098091E10057
:101BF00083FF29C08091E20083FF25C08091E1002E
:101C0000877F8093E10082E08093F1011092ED01E3
:101C10008091E1008E7F8093E1008091E2008E7FD1
:101C20008093E2008091E20080618093E20042E0D4
:101C300060E080E00E94610C8091F00088608093F9
:101C4000F0000E94D509FF91EF91BF91AF919F9154
:101C50008F917F916F915F914F913F912F910F9055
:101C60000FBE0F901F9018951F920F920FB60F92F4
:101C700011242F933F934F935F936F937F938F9391
:101C80009F93AF93BF93CF93DF93EF93FF93C09155
:101C9000E900CF708091EC00D82FD17080FDD0E8A2
:101CA0001092E9008091F000877F8093F000789493
:101CB0000E94780E1092E9008091F0008860809375
:101CC000F000CD2BCF70C093E900FF91EF91DF9131
:101CD000CF91BF91AF919F918F917F916F915F91C4
:101CE0004F913F912F910F900FBE0F901F9018951D
:101CF0001F93CF93DF93CDB7DEB7AA970FB6F894B3
:101D0000DEBF0FBECDBFE2EFF1E088E08E0F909115
:101D1000F10091938E13FBCF0E94F4098091E800AB
:101D200083FF1FC18091F2019091F301492F50E090
:101D30004A30510508F015C1FA01EA5AFF4F0C94D8
:101D4000B323803881F0823809F00BC18091F6010D
:101D50008F708093E9008091EB0085FB882780F9E4
:101D60001092E90006C08091EE019091EF0191116F
:101D700082609091E800977F9093E8008093F10053
:101D80001092F100C8C0282F2D7F09F0EAC08823E7
:101D900019F0823061F0E5C08091F401813009F0E2
:101DA000E0C0933009F080E08093EF012BC0809178
:101DB000F401811127C08091F6018F7009F4D1C020
:101DC0008093E9002091EB0020FF1CC0933021F4A8
:101DD0008091EB00806214C09091EB009061909331
:101DE000EB0021E030E0A90102C0440F551F8A95A5
:101DF000E2F74093EA001092EA008091EB008860DD
:101E00008093EB001092E9008091E800877F86C004
:101E10008111A7C01091F4011F778091E3008078B1
:101E2000812B8093E3008091E800877F8093E80016
:101E30000E94960C8091E80080FFFCCF8091E30027
:101E400080688093E300111102C082E001C083E04A
:101E50008093F10186C08058823008F082C0809162
:101E6000F4019091F5018C3D53E0950779F583E0FD
:101E70008A838AE289834FB7F894DE01139620E0C3
:101E80003EE051E2E32FF0E050935700E49120FF51
:101E900003C0E295EF703F5FEF708E2F90E0EA3065
:101EA00010F0C79601C0C0968D939D932F5F24318B
:101EB00049F74FBF8091E800877F8093E8006AE28E
:101EC00070E0CE0101960E949D0B14C0AE014F5FE1
:101ED0005F4F6091F6010E94E40ABC01009709F48B
:101EE00040C09091E800977F9093E80089819A81A3
:101EF0000E94000C8091E8008B778093E80031C04D
:101F0000803879F58091E800877F8093E8008091A0
:101F1000ED018093F1008091E8008E778093E800D6
:101F20000E94960C1EC081111CC09091F401923049
:101F3000C0F48091E800877F8093E8009093ED01E2
:101F40000E94960C8091ED01811106C08091E30002
:101F500087FD02C081E001C084E08093F1010E940E
:101F6000E0098091E80083FF0AC08091E800877F44
:101F70008093E8008091EB0080628093EB00AA964A
:101F80000FB6F894DEBF0FBECDBFDF91CF911F918A
:101F900008950895CF938091F1018823A1F0C09115
:101FA000E900CF709091EC00892F817090FD80E85E
:101FB000C82B1092E9008091E80083FD0E94780E02
:101FC000CF70C093E900CF910895909375018093ED
:101FD00074010895E0917401F0917501309721F03A
:101FE0000190F081E02D099480E00895E091740162
:101FF000F0917501309721F00280F381E02D099472
:102000000895E0917401F0917501309721F00480FA
:10201000F581E02D099408952091720130917301AA
:102020008217930771F09093730180937201E0918E
:102030007401F0917501309721F00680F781E02D51
:1020400009940895209170013091710182179307CE
:1020500071F09093710180937001E0917401F0919F
:102060007501309721F00084F185E02D09940895E1
:1020700008950C9438100E94921B0E9433030C9414
:10208000541C9F92AF92BF92CF92DF92EF92FF9239
:102090000F931F93CF93DF9300D000D000D0CDB724
:1020A000DEB70E944B030DE010E0AA24A394B12CEC
:1020B000902E802F0E943904980129583E4F6901C3
:1020C000F901F080F826A1F40150110988F78FEF8B
:1020D00089838A831B820E949B1B8160782F9D834A
:1020E0008C8349815A816B818D810E94D8102FC0C9
:1020F0009091DA0191FF04C08E830E943F048E818B
:1021000025E030E0A501022E01C0440F0A94EAF751
:10211000E42E4F21C1F029839A828E2191E009F4A7
:1021200090E09B830E949B1B8160782F9D838C8312
:1021300049815A816B818D810E94D810F60180817E
:10214000E826E08204C021503109E0F6BDCF0E94AC
:102150003B1F109176010E94EA0F1817B9F00E94F8
:10216000EA0F8093760126960FB6F894DEBF0FBE75
:10217000CDBFDF91CF911F910F91FF90EF90DF9036
:10218000CF90BF90AF909F900C94E30826960FB627
:10219000F894DEBF0FBECDBFDF91CF911F910F919D
:1021A000FF90EF90DF90CF90BF90AF909F900895F9
:1021B000CF93DF93CDB7DEB72B970FB6F894DEBF82
:1021C0000FBECDBF4F83588769877A878B87DE0123
:1021D000119686E0FD0111928A95E9F785E0FE01EE
:1021E000379601900D928A95E1F749815A816B816A
:1021F0007C818D819E810E9421172B960FB6F894C9
:10220000DEBF0FBECDBFDF91CF910895CF9388235E
:1022100009F4C2C0C82F823859F40E94EA0F81FD28
:10222000BBC089E30E94FB190E94C81A89E30CC055
:10223000833879F40E94EA0F80FDAEC083E50E94E6
:10224000FB190E94C81A83E50E943D1ACF910C9495
:10225000C81A843859F40E94EA0F82FD9DC087E4B1
:102260000E94FB190E94C81A87E4EECF8CEF8C0FF6
:10227000813A48F48C2F0E947E2181118DC08C2FD1
:102280000E94FB19E3CF80E28C0F883048F4C770BE
:1022900081E001C0880FCA95EAF70E94811AD6CF63
:1022A0008BE58C0F833078F4C53A29F0C63A31F0CB
:1022B00083E890E005C081E890E002C082E890E009
:1022C000CF910C940C1088E58C0F833108F064C01A
:1022D000C83A39F1C93A41F1CA3A49F1CB3A51F118
:1022E000CC3A59F1CD3A61F1C03B69F1CE3A71F186
:1022F000CF3A79F1C13B81F1C23B89F1C33B91F106
:10230000C43B99F1C53BA1F1C63BA9F1C73BB1F173
:10231000C83BB9F1C93BC1F1CA3BC9F180E090E0CB
:1023200038C082EE90E035C089EE90E032C08AEE8F
:1023300090E02FC085EB90E02CC086EB90E029C0A8
:1023400087EB90E026C08CEC90E023C08DEC90E011
:1023500020C083E891E01DC08AE891E01AC082E9BC
:1023600091E017C084E991E014C081E292E011C0CD
:1023700083E292E00EC084E292E00BC085E292E03C
:1023800008C086E292E005C087E292E002C08AE2DD
:1023900092E0CF910C942210CF910895882309F4F4
:1023A0004BC0823859F40E94EA0F81FF45C089E38F
:1023B0000E94FB190E94C81A89E30CC0833871F48B
:1023C0000E94EA0F80FF38C083E50E94FB190E943B
:1023D000C81A83E50E943D1A0C94C81A843859F42F
:1023E0000E94EA0F82FF28C087E40E94FB190E9426
:1023F000C81A87E4EFCF9CEF980F913A58F390E218
:10240000980F983050F4877091E001C0990F8A9529
:10241000EAF7892F0E94871ADFCF9BE5980F933048
:1024200020F480E090E00C940C10885A833120F462
:1024300080E090E00C9422100895882321F00E94FF
:10244000811A0C94C81A0895882321F00E94871AD3
:102450000C94C81A08957F928F929F92AF92BF9268
:10246000CF92DF92EF92FF920F931F93CF93DF9360
:102470001F92CDB7DEB77C01C62E772EFC010581F9
:1024800002950F70128111110E949E1A0E94F41978
:10249000882379F0112369F080E28C0D883048F0B0
:1024A00082E00E94DD190E94F41991E0D82ED9260D
:1024B00001C0D12CE72DE295EF70F0E0E05AFF4F1C
:1024C0000C94B323872D807F072D0F70882311F084
:1024D0000295007F112389F0002309F490C180E266
:1024E0008C0D883020F4802F0E94811A03C0802F29
:1024F0000E94911A0E94C81A82C18C2D0E94CE118E
:10250000002309F495C180E28C0D883020F4802FDF
:102510000E94871A03C0802F0E94971A0E94C81A2F
:1025200087C1972D907F872D8F70903211F0829503
:10253000807FCC2021F0F1E0CF16B1F01EC0112336
:1025400049F0002309F414C1013009F011C10E94BF
:10255000B11A6EC1002319F0013009F469C18983F1
:102560000E94B41A89810AC1112321F0023008F0B7
:102570005FC1FEC001115CC101C1112321F0002324
:1025800009F4F6C03CC1002309F4F8C03EC1872D10
:1025900086958695837090E0009719F0019761F019
:1025A00047C1112321F08C2D972D937002C080E03C
:1025B00090E00E940C103CC1112321F08C2D972D2E
:1025C000937002C080E090E00E94221031C18C2DF7
:1025D000112319F00E94431E02C00E94AB1E0E94EC
:1025E000301F26C1872D837009F052C0111120C100
:1025F0008C2D829586958770880F880F9C2D9F70F3
:10260000892E912CA12CB12C082E04C0880C991C69
:10261000AA1CBB1C0A94D2F7C4FE14C00FE010E041
:1026200020E030E0B901A80104C0440F551F661F27
:10263000771F8A95D2F7CB01BA0160957095809586
:10264000909503C060E070E0CB01272D269526957C
:10265000237030E02230310569F02330310589F0F4
:10266000682979298A299B292130310571F00E9436
:102670006918DEC0682979298A299B290E94851852
:10268000D7C00E946918C501B4010E944D18D0C07E
:10269000112319F0872D817001C08695882309F4D4
:1026A000C7C08C2D829586958770880F880F9C2DCA
:1026B0009F70892E912CA12CB12C082E04C0880C5F
:1026C000991CAA1CBB1C0A94D2F7C4FE14C00FE0CC
:1026D00010E020E030E0B901A80104C0440F551F0C
:1026E000661F771F8A95D2F7CB01BA016095709566
:1026F0008095909503C060E070E0CB01272D269572
:1027000026952370422F50E04230510569F0433046
:10271000510589F0682979298A299B294130510579
:1027200071F00E94431984C0682979298A299B295C
:102730000E945F197DC00E944319C501B4010E9427
:10274000271976C08C2D90E0FC01E05EF109E5319F
:10275000F10508F050C0E059FF4F0C94B3230C2D45
:102760000F70872D8F71112331F00E94C018802FB8
:102770000E941D125DC00E94E118802F0E94241249
:1027800057C0112339F0011153C0872D8F710E945A
:1027900006194EC0023008F04BC0F7CF112339F0B4
:1027A000872D8F710E94C01843C01123C9F3872D54
:1027B0008F710E94E1183CC0112329F0872D8F7181
:1027C0000E94AB1835C00E94A11832C0112351F0ED
:1027D000172D1F71812F0E94C01863E0812F0E9466
:1027E000D41926C081E00E94DD19023008F182E090
:1027F0000E94DD191DC0112331F0002389F28C2DB8
:102800000E94061115C0002391F28C2D0E94CE115A
:102810000FC0472D4F706C2DC7010E9415050E94F7
:10282000C51706C0472D4F706C2DC7010E94F205D9
:10283000DD20F9F00E94D01980FD1BC0F701128243
:102840000E94CA190E94C018C7010E9448140E9421
:10285000CA190F90DF91CF911F910F91FF90EF90C8
:10286000DF90CF90BF90AF909F908F907F900C940F
:10287000E1180F90DF91CF911F910F91FF90EF9092
:10288000DF90CF90BF90AF909F908F907F900895F2
:102890000F931F93CF93DF93EC01888199812B8154
:1028A0003C81232BB9F09F3F11F48F3F99F0CE016B
:1028B0000E944A05882371F0688179818A810E948B
:1028C000C6198C010E947B190E944218B801CE01E2
:1028D0000E942B12DF91CF911F910F9108950E94BA
:1028E0009E1A0E94AE1A0E94731A0E94C81A0E9471
:1028F000E11F0E94301F80E090E00E940C1080E0F9
:1029000090E00C9422100E948E1A0C946F140E9476
:10291000BB19292F22952F7030E02C3031054CF453
:102920002A3031056CF42250310922303105A8F4E7
:1029300007C02C30310569F02F30310551F00DC042
:10294000803F69F018F4803E40F409C0843F29F4C8
:1029500006C093FB882780F9089580E0089581E000
:102960000895CF93DF9300D000D01F92CDB7DEB78C
:102970000F900F900F900F900F90DF91CF910895CF
:10298000CF93DF9300D000D000D0CDB7DEB726962E
:102990000FB6F894DEBF0FBECDBFDF91CF91089583
:1029A0001F93CF93DF93C091850116E0809186013C
:1029B000C81799F0D0E01C9FF0011D9FF00D112465
:1029C000E957FE4F408151816281738184819581F5
:1029D0000E94C0142196C770E9CFDF91CF911F915B
:1029E00008954091B7015091B8016091B90170917B
:1029F000BA018091BB019091BC010C94C0148091EC
:102A0000BC0182958F7009F054C08091B901882370
:102A100009F44FC080918501A09186016091B701B2
:102A20007091B8014091BA015091BB01B6E08A178C
:102A300009F43FC090E041155105C1F17F3F11F409
:102A40006F3FA1F1B89FF001B99FF00D1124E95734
:102A5000FE4F218172132AC02081621327C0228178
:102A6000211124C0238134812417350710F421500B
:102A70003109241B350B283C3105C0F42091BC01E1
:102A80002F7020612093BC0126E0289FF001299F30
:102A9000F00D1124E457FE4F80818F708061808398
:102AA00087EB91E00E9448140C94D0140196877033
:102AB000BECF0895CF92DF92EF92FF920F931F93B4
:102AC000CF93DF93CDB7DEB762970FB6F894DEBF32
:102AD0000FBECDBF8C0185E0F801DE011D9601908F
:102AE0000D928A95E1F7D8014C9111965C9111975E
:102AF00012966C9112971396CD90DC9014973091AA
:102B0000B7017091B8018091BA019091BB01009713
:102B100009F46BC17F3F19F43F3F09F466C1E090AF
:102B2000B901EE2009F4C0C02091BC01C816D90635
:102B300028F0F601E81BF90BCF0104C080959095B1
:102B40008C0D9D1DFF24F394883C910578F0F12CA9
:102B5000207F09F0C6C07C2DD98AC88A89890E9445
:102B6000B11487EB91E00E944814B1C0822F807F9E
:102B700009F046C0751314C0341312C0611110C09F
:102B80002F7020612093BC010E94F11487EB91E02B
:102B90000E9448148091BC01D80115968C932EC0D8
:102BA000CD2819F15F3F11F44F3FF9F0F62E611176
:102BB0001CC0809185012091860136E0821709F4BE
:102BC0005AC090E0389FF001399FF00D1124E95769
:102BD000FE4F7181571306C07081471303C0728185
:102BE000711103C001968770E9CFF62E662309F4B0
:102BF00018C18091BC0181608093BC01F12C11C18E
:102C0000751308C0341306C0611104C08091BC0163
:102C1000D801C3C04D875E878D859E856A8B0E94D3
:102C200087146A898823E1F16623D1F12091BC01E0
:102C3000822F82958F7090E0029774F08091B70197
:102C40009091B80198878F831986DB86CA862C8776
:102C5000CE0107960E94481486E0F801A7EBB1E088
:102C600001900D928A95E1F70E94FF140E94F114E1
:102C7000FF24F394D6C04D875E878D859E850E9484
:102C8000BB19292F22952F7030E0223031050CF02E
:102C9000BCC09F7009F0B6C0805E883008F4C1C027
:102CA000C8010E944814E4CFC816D90608F453C0DE
:102CB000F601E81BF90BCF01883C910508F450C0E0
:102CC000F12C7C2DD98AC88A89890E94B114E7EB3E
:102CD000F1E086E0DF011D928A95E9F70E94F11488
:102CE000A0C0751314C0341312C0611110C08091BC
:102CF000BC01F8018583C8010E94481486E0E7EB17
:102D0000F1E0DF011D928A95E9F7FE2C8AC04D871C
:102D10005E878D859E856A8B0E9487146A898823C9
:102D200009F4BECF662309F4BBCF2091BC01822FEA
:102D300082958F7090E002970CF48ECF8091B7014E
:102D40009091B8019A8389831B82DD82CC822E8385
:102D5000CE0101967FCF809590958C0D9D1DACCFB7
:102D6000F62E662309F49CCF75132EC034132CC0A5
:102D70002091BC0120FD1FC0822F82958F70D9F059
:102D8000D80115962C9315978F3049F08F5F982FA7
:102D90009295907F822F8F70892B15968C93C80106
:102DA0000E94481486E0F801A7EBB1E001900D9273
:102DB0008A95E1F793CF86E0F801A7EBB1E00190A7
:102DC0000D928A95E1F72DC04D875E878D859E8592
:102DD0000E948714811140CF8091BC018160809353
:102DE000BC01C8010E9448141CC0662309F458CFD6
:102DF0004D875E878D859E850E948714882309F400
:102E00004FCF2ACF811148CF0CC0243031050CF0B0
:102E100047CF9F7009F440CFF8019581907F09F06A
:102E20003BCF8F2D62960FB6F894DEBF0FBECDBF9D
:102E3000DF91CF911F910F91FF90EF90DF90CF9096
:102E400008951F93CF93DF93CDB7DEB72C970FB6BE
:102E5000F894DEBF0FBECDBF4F83588769877A874E
:102E60008B879C87CE0107960E945A15882369F0AC
:102E70008F8198852A853B85232BF1F19F3F09F0AF
:102E800063C08F3F09F060C037C086E0FE0137960F
:102E9000DE01119601900D928A95E1F76F81788598
:102EA000EA85FB85309741F17F3F11F46F3F21F1B7
:102EB0002091860130E0C9010196877099274091E1
:102EC000850150E08417950709F447C069837A8328
:102ED000FD83EC8396E0929FD001939FB00D112467
:102EE000A957BE4FFE01319601900D929A95E1F7D8
:102EF000809386010E94D01416E080918501909104
:102F000086018917C1F1189FC001112489579E4F6E
:102F10000E945A15882379F1E09185011E9FF001E6
:102F20001124E957FE4F4081518162817381848170
:102F300095810E94C0148091850190E00196877070
:102F4000992780938501D9CF4F81588569857A85E6
:102F50008B859C850E94C014CFCF0E948314109251
:102F6000860110928501E7EBF1E086E0DF011D921A
:102F70008A95E9F7C1CF2C960FB6F894DEBF0FBE45
:102F8000CDBFDF91CF911F910895EF92FF920F93E4
:102F90001F93CF93DF938C01009709F46CC0F12C41
:102FA000EE24E394E8012196F8018491843740F4FB
:102FB000843008F051C0813081F0823019F15BC05B
:102FC000853709F444C0A8F19CE7980F903708F0C2
:102FD00052C08F770E94CE1141C00E5F1F4FFE017D
:102FE000C49180E28C0F883048F4C7708E2D01C0E8
:102FF000880FCA95EAF70E94A11A14C08C2F0E946C
:1030000006112DC00E5F1F4FFE01C49180E28C0F90
:10301000883058F4C7708E2D01C0880FCA95EAF722
:103020000E94A71A0E94C81A1AC08C2F0E94CE11A3
:1030300016C00E5F1F4FFE01C491CC2381F08FE9B3
:103040009FE00197F1F700C00000C150F6CF0E5F7E
:103050001F4FFE01F49003C00E9406118E018F2DB8
:10306000882309F49FCFEFE9FFE03197F1F700C023
:1030700000008150F5CFDF91CF911F910F91FF900C
:10308000EF90089508956093C1017093C2018093F9
:10309000C3019093C4010C946F140F931F9300917C
:1030A000C1011091C2012091C3013091C401DC0122
:1030B000CB01802B912BA22BB32B8093C10190933A
:1030C000C201A093C301B093C4011F910F910C944E
:1030D0006F140F931F930091C1011091C2012091B1
:1030E000C3013091C401DC01CB0180239123A223D1
:1030F000B3238093C1019093C201A093C301B09305
:10310000C4011F910F910C946F140F931F930091A2
:10311000C1011091C2012091C3013091C401DC01B1
:10312000CB0180279127A227B3278093C1019093D9
:10313000C201A093C301B093C4011F910F910C94DD
:103140006F141092BD011092BE011092BF01109237
:10315000C0010C946F1441E050E060E070E004C0E6
:10316000440F551F661F771F8A95D2F74093BD0104
:103170005093BE016093BF017093C0010C946F1413
:1031800041E050E060E070E004C0440F551F661F4E
:10319000771F8A95D2F78091BD019091BE01A091D1
:1031A000BF01B091C001482B592B6A2B7B2B409358
:1031B000BD015093BE016093BF017093C0010C9498
:1031C0006F1441E050E060E070E004C0440F551F10
:1031D000661F771F8A95D2F7409550956095709538
:1031E0008091BD019091BE01A091BF01B091C0013D
:1031F000482359236A237B234093BD015093BE018A
:103200006093BF017093C0010C946F1441E050E0D3
:1032100060E070E004C0440F551F661F771F8A9559
:10322000D2F78091BD019091BE01A091BF01B091F4
:10323000C001482759276A277B274093BD01509337
:10324000BE016093BF017093C0010C946F140F9383
:103250001F930091BD011091BE012091BF013091DB
:10326000C001DC01CB01802B912BA22BB32B8093CF
:10327000BD019093BE01A093BF01B093C0011F9107
:103280000F910C946F140F931F930091BD01109137
:10329000BE012091BF013091C001DC01CB01802330
:1032A0009123A223B3238093BD019093BE01A093E9
:1032B000BF01B093C0011F910F910C946F140F9335
:1032C0001F930091BD011091BE012091BF0130916B
:1032D000C001DC01CB0180279127A227B32780936F
:1032E000BD019093BE01A093BF01B093C0011F9197
:1032F0000F910C946F140895CF92DF92EF92FF928A
:103300000F931F93CF93DF938C01C090C101D09096
:10331000C201E090C301F090C4018091BD01909181
:10332000BE01A091BF01B091C001C82AD92AEA2AE2
:10333000FB2ACFE1D0E0D701C6010C2E04C0B69520
:10334000A795979587950A94D2F780FF06C0B80194
:103350008C2F0E944808019721F4219760F780E0A4
:1033600001C08C2FDF91CF911F910F91FF90EF90B3
:10337000DF90CF900895CF93DF93EC010E947C19EA
:10338000BE010E944808DF91CF910895CB010E94B1
:10339000BB1908958091C5018595859585950895FA
:1033A0008091C5018770089598E0899F900111244C
:1033B000262B2093C5010C94C0182091C50180953F
:1033C00082238093C501982F977069F430E0482FCD
:1033D000552747FD50952417350729F08595859584
:1033E00085950C94E11808959091C501977081E03E
:1033F00009F480E0089590910C01992321F09091B7
:103400000D01911109C020910E0130910F01F901B8
:1034100032969FEF40E01FC0982F9695969596950F
:103420009F3050F5E0910E01F0910F01E90FF11D71
:10343000877021E030E0A90102C0440F551F8A9532
:10344000E2F7CA019181892B818308959F3F39F06A
:103450004F5F4E3041F051915813F8CF0DC05111CC
:10346000F7CF942FF5CF9F3F39F0F901E90FF11D08
:1034700097FDFA9582830895089590910C01992300
:1034800021F090910D01911109C020910E01309110
:103490000F01F9013296205F3F4F1FC0982F96957C
:1034A000969596959F30F0F4E0910E01F0910F0102
:1034B000E90FF11D877021E030E0A90102C0440F3F
:1034C000551F8A95E2F7CA018095918189238183EE
:1034D00008953196E217F30729F090819813F9CFF8
:1034E0001082F7CF089581E090E0E0910E01F09115
:1034F0000F01E80FF91F1082019680319105A9F79D
:1035000008959091D901892B8093D90108958095D0
:103510009091D90189238093D90108951092D901FE
:1035200008959091D801892B8093D80108958095B2
:103530009091D80189238093D80108951092D801E1
:1035400008959091D701892B8093D7010895809594
:103550009091D70189238093D70108951092D701C4
:1035600008958093C60108951092C6010895809130
:103570000E0190910F01FC0131969C01205F3F4F9D
:1035800080E0919191118F5FE217F307D1F70895D1
:10359000E0910E01F0910F018091D9018083E091BB
:1035A0000E01F0910F0190818091D801892B8083C9
:1035B000E0910E01F0910F0190818091D701892B4C
:1035C00080838091C601882361F0E0910E01F09123
:1035D0000F019081892B80830E94B71A811110926C
:1035E000C60180910E0190910F010C94F60F20E01E
:1035F000009739F0AC0141505109842395232F5F86
:10360000F7CF822F0895CF92DF92EF92FF926C0155
:10361000EE24FF24C114D104E104F10421F0C70118
:10362000B60120E101C020E0C72ED82EE92EFF24EC
:10363000C114D104E104F10419F0285FC701B601F7
:103640006B017C0154E0F694E794D794C7945A95A3
:10365000D1F7C114D104E104F10419F02C5FC701C2
:10366000B6016B017C0142E0F694E794D794C794CD
:103670004A95D1F7C114D104E104F10419F02E5F89
:10368000C701B601DC01CB01B695A7959795879543
:10369000892B8A2B8B2B09F02F5F822FFF90EF90C5
:1036A000DF90CF9008958091F101843021F1109244
:1036B000DB0120E488E190E00FB6F894A8958093B0
:1036C00060000FBE2093600080E00E94E30883B793
:1036D000817F846083BF83B7816083BF789488953E
:1036E00083B78E7F83BF88E10FB6F8948093600024
:1036F000109260000FBE0895089508950E947C1BEB
:103700000E944B030E947D1B0E94400491E08111A6
:1037100001C090E0892F08950E9483140E94EA0F4F
:103720000C94E30882E084BD93E095BD9AEF97BDC9
:1037300080936E0008952FB7F8948091DC019091EA
:10374000DD01A091DE01B091DF012FBF0895CF927E
:10375000DF92EF92FF920F931F932FB7F89440914F
:10376000DC015091DD016091DE017091DF012FBF1E
:103770006A017B01EE24FF248C0120E030E0C016BA
:10378000D106E206F30610F4415051099A01281BB4
:10379000390BC9011F910F91FF90EF90DF90CF90EF
:1037A00008951F920F920FB60F9211248F939F933B
:1037B000AF93BF938091DC019091DD01A091DE0178
:1037C000B091DF010196A11DB11D8093DC019093A2
:1037D000DD01A093DE01B093DF01BF91AF919F9116
:1037E0008F910F900FBE0F901F9018950E94E70CBD
:1037F000F8942FEF87EA91E6215080409040E1F75E
:1038000000C0000087E090EBDC018093FB01909307
:10381000FC01A093FD01B093FE019CE088E10FB68E
:10382000F894A895809360000FBE90936000FFCF3E
:10383000EF92FF920F931F93CF93DF93D82FCDE09A
:103840008C2F0E94390405E010E0E82EF12CC7010E
:10385000002E02C0959587950A94E2F780FF09C073
:10386000602F7C2F80E00E94F305D81302C081E016
:1038700006C00150110958F7C15010F780E0DF91E0
:10388000CF911F910F91FF90EF900895CF93C82F84
:103890008CE20E94181C882321F08C2FCF910C946D
:1038A000181C80E0CF910895CF930E949B1D811139
:1038B00002C00E94811DC5E6C15049F00E944B0321
:1038C0008FE39CE90197F1F700C00000F5CF89E292
:1038D0000E94461C811113C18AE20E94461C81117C
:1038E0000E94811D85E00E94461C81110E94F61BEA
:1038F0000E94A61D8093DA0187E00E94461C88235F
:10390000A9F18BE10E94461C882351F08091DA01D5
:1039100081FB222720F991E0922790FB81F90EC0CC
:103920008EE00E94461C882361F08091DA0182FBC0
:10393000222720F991E0922790FB82F98093DA0107
:1039400015C080E10E94461C9091DA01882341F065
:1039500093FB222720F981E0822780FB93F904C0A2
:10396000892F809580FB90F99093DA018091DA019C
:103970000E94AA1D0E94B81D8093FA0180EE0E9449
:10398000461C882341F08091FA01982F909590FB76
:1039900080F98093FA0189E30E94461C882359F03C
:1039A0008091FA0181FB222720F991E0922790FB78
:1039B00081F98093FA0182EE0E94461C882359F017
:1039C0008091FA0182FB222720F991E0922790FB57
:1039D00082F98093FA0186EE0E94461C882359F0F2
:1039E0008091FA0183FB222720F991E0922790FB36
:1039F00083F98093FA0183EE0E94461C882359F0D4
:103A00008091FA0184FB222720F991E0922790FB14
:103A100084F98093FA0185E30E94461C882359F0BB
:103A20008091FA0185FB222720F991E0922790FBF3
:103A300085F98093FA0181E30E94461C882359F09E
:103A40008091FA0186FB222720F991E0922790FBD2
:103A500086F98093FA0181E10E94461C882359F07F
:103A60008091FA0187FB222720F991E0922790FBB1
:103A700087F98093FA018091FA010E94BC1D809120
:103A8000FA0187FB882780F980930D0187E20E9465
:103A9000461CC82F8EE10E94461C8111C2608FE136
:103AA0000E94461C8111C46080E20E94461C811164
:103AB000C86081E20E94461C8111C06182E20E94BE
:103AC000461C8111C06283E20E94461C8111C064C1
:103AD00084E20E94461C882311F0C06802C0CC23F7
:103AE00029F08C2F0E94B31D6C2F03C00E94AF1DC4
:103AF000682F70E080E090E0CF910C944318CF9154
:103B000008956DEE7EEF80E090E00E94ED2360E08E
:103B100082E090E00E94DB2360E083E090E00E947E
:103B2000DB2360E084E090E00E94DB2360E085E03E
:103B300090E00C94DB2380E090E00E94D52321E00C
:103B40008D3E9E4F09F020E0822F089582E090E0A4
:103B50000C94CD23682F82E090E00C94DB2383E06B
:103B600090E00C94CD23682F83E090E00C94DB234D
:103B700084E090E00C94CD23682F84E090E00C94D6
:103B8000DB238091E20180FF0BC06091130185E08F
:103B9000689FB001112475956795759567952BC041
:103BA00081FF09C06091130185E0689FB001112475
:103BB0007595679520C082FF07C06091130185E06D
:103BC000689FB001112417C09091E3019923D1F0AF
:103BD00060911201961788F72091130185E0289FC4
:103BE00090011124929FA001939F500D112470E029
:103BF000CA010E949F236038710540F46115710568
:103C000039F002C065E070E0862F08958FE70895CF
:103C100081E008958091E20180FF08C06091110168
:103C200070E0759567957595679521C081FF06C011
:103C30006091110170E07595679519C082FF04C00D
:103C40006091110170E010C09091E3019923C1F0DF
:103C5000609110019617A0F780911101899FC00112
:103C6000112470E00E949F236038710528F46115CB
:103C7000710521F0862F08958FE7089581E008955A
:103C800061E070E0F4CF803F21F40E94C11D819576
:103C900004C0813F29F40E94C11D8093E60108956C
:103CA000823F21F40E94C11D819504C0833F29F405
:103CB0000E94C11D8093E5010895893F19F40E9477
:103CC0000A1E05C08A3F31F40E940A1E8195809326
:103CD000E70108958B3F21F40E940A1E819504C0DC
:103CE0008C3F29F40E940A1E8093E8010895843FC6
:103CF00021F48091E401816017C0853F21F4809117
:103D0000E401826011C0863F21F48091E401846067
:103D10000BC0873F21F48091E401886005C0883F93
:103D200031F48091E40180618093E40108958D3F36
:103D300021F48091E20181600BC08E3F21F48091DB
:103D4000E201826005C08F3F29F48091E201846026
:103D50008093E2010895803F39F48091E60187FF66
:103D60006CC01092E60169C0813F29F48091E601A0
:103D70001816BCF362C09091E501823F29F497FFC9
:103D80005CC01092E50159C0833F19F41916CCF3B9
:103D900054C0893F41F48091E70118160CF04DC0E2
:103DA0001092E7014AC08A3F29F48091E70187FF1A
:103DB00044C0F6CF8B3F39F48091E80187FF3DC0C6
:103DC0001092E8013AC08C3F29F48091E80118165E
:103DD000BCF333C0843F21F48091E4018E7F17C08F
:103DE000853F21F48091E4018D7F11C0863F21F44D
:103DF0008091E4018B7F0BC0873F21F48091E40127
:103E0000877F05C0883F31F48091E4018F7E8093E5
:103E1000E40113C08D3F21F48091E2018E7F0BC03D
:103E20008E3F21F48091E2018D7F05C08F3F29F400
:103E30008091E2018B7F8093E2018091E501811105
:103E40000EC08091E60181110AC08091E7018111C5
:103E500006C08091E801811102C01092E30108952B
:103E600084EE91E00E9401100E949B1B9093E1015F
:103E70008093E00108951F93CF93DF938091E00139
:103E80009091E1010E94A71BAC019091E30199235D
:103E900021F02091140130E006C0209115018AE044
:103EA000289F900111244217530708F486C080917F
:103EB000E501C091E601D091E7011091E80181117F
:103EC00007C0C11176C0D11174C0111172C075C084
:103ED0009F3F19F09F5F9093E301181624F40E940E
:103EE000C11D8093E5018091E50187FF05C00E9417
:103EF000C11D81958093E5011C1624F40E94C11D0B
:103F00008093E6018091E60187FF05C00E94C11DF4
:103F100081958093E6016091E501662339F1C091B6
:103F2000E601CC2319F1772767FD7095872F972F2E
:103F30000E94B02223E333E343E35FE30E941423B0
:103F40000E947D226093E5016C2F772767FD7095B5
:103F5000872F972F0E94B02223E333E343E35FE3ED
:103F60000E9414230E947D226093E6011D1624F412
:103F70000E940A1E8093E7018091E70187FF05C038
:103F80000E940A1E81958093E701111624F40E9475
:103F90000A1E8093E8018091E80187FF05C00E9416
:103FA0000A1E81958093E801DF91CF911F910C94B7
:103FB000301F9F3F09F08ECF96CFDF91CF911F9199
:103FC0000895E4EEF1E085E0DF011D928A95E9F7BE
:103FD0001092E3011092E2010895833081F128F4F8
:103FE000813059F08230D1F00895853009F449C00C
:103FF000B8F1863009F456C0089580911501262F36
:1040000030E0280F311D2F3F310524F4680F6093F5
:10401000150108958FEF8093150108958091140183
:10402000262F30E0280F311D2F3F310524F4680F73
:104030006093140108958FEF809314010895809187
:104040001301262F30E0280F311D2F3F310524F4B6
:10405000680F6093130108958FEF80931301089503
:1040600080911201262F30E0280F311D2F3F31059E
:1040700024F4680F6093120108958FEF809312016A
:10408000089580911101262F30E0280F311D2F3F18
:10409000310524F4680F6093110108958FEF809328
:1040A0001101089580911001262F30E0280F311D55
:1040B0002F3F310524F4680F6093100108958FEFAE
:1040C000809310010895833011F128F4813049F074
:1040D000823091F00895853081F120F18630C1F170
:1040E000089580911501681720F4861B80931501AF
:1040F000089510921501089580911401681720F415
:10410000861B8093140108951092140108958091E4
:104110001301681720F4861B8093130108951092F1
:104120001301089580911201681720F4861B809373
:1041300012010895109212010895809111016817DB
:1041400020F4861B809311010895109211010895A7
:1041500080911001681720F4861B80931001089548
:104160001092100108950F931F938D3109F46BC0C5
:1041700008F03FC08E3009F47FC0C0F4873009F4E6
:1041800069C068F4863009F0B1C08091DA01817F9E
:104190008E7F8093DA0181E08093EA01A8C08830A5
:1041A00009F4A2C08B3009F49FC0A0C0863109F485
:1041B0009BC078F4803109F472C0813109F096C057
:1041C0000E94831490910D0181E0892780930D0155
:1041D0008BC0893109F488C08B3109F087C0809188
:1041E000DA0181FB222720F991E0922790FB81F9E7
:1041F0004CC0853309F470C048F4873209F46CC0B0
:1042000008F459C0893209F467C070C0833438F4A7
:104210008A3308F04EC0883309F466C067C083341F
:1042200009F45AC0883409F061C00E9483140FEF6A
:1042300013ED20E3015010402040E1F700C00000E2
:104240000E94F61B51C00E9437220E94EA0F0E9472
:10425000E3084AC09091DA01892F8095817080FB34
:1042600090F929F0966098609093DA0140C0997FA8
:10427000977F9093DA0138C08091DA0182FB222780
:1042800020F991E0922790FB82F98093DA0199233B
:1042900059F18091DA0181608093DA0125C0809123
:1042A000DA0183FB222720F991E0922790FB83F922
:1042B000ECCF895301C08D5141E050E060E070E0E7
:1042C0008A019B0104C0000F111F221F331F8A9512
:1042D000D2F7C901B80104C061E070E080E090E06D
:1042E0000E9443180E94831481E001C080E01F9166
:1042F0000F91089580E0089580E00895CF93C82F2E
:104300008091EA01813079F018F08230E9F187C0BC
:10431000E0910E01F0910F018081813169F08232CC
:1043200009F07FC009C0E0910E01F0910F0180817A
:10433000813111F0823261F48C2F0E947A21811137
:1043400004C08C2F0E94B3201DC081E090E01AC0F1
:104350008C2F0E947C21811114C0C43179F048F463
:10436000CB3079F0C03109F060C082E08093EA017F
:1043700008C0C93219F0C83321F057C01092EA01C1
:1043800054C081E0817053C0C93289F118F5C4313D
:1043900071F1A8F4C73009F046C08AE08093150196
:1043A00094E19093140193E0909313018093120190
:1043B00088E08093110188E28093100134C0CE51CF
:1043C000C63088F5EC2FF0E0E65DFE4F80818093EB
:1043D000E90129C0CE34E9F020F4CB3421F56AE0BC
:1043E00013C0C13579F0C235F1F461E00DC08091A0
:1043F000E901882319F01092E90115C081E080934A
:10440000EA0115C061E006C08091E9010E94ED1F3C
:104410000AC06AE08091E9010E94632004C0109202
:10442000EA0180E004C081E002C080E0ABCFCF9120
:104430000895E1E8F0E08081886080838081816078
:1044400080838FB7F89493E09093890090ED9093D8
:1044500088008FBF0895EFE6F0E08081826080835E
:104460000895EFE6F0E080818D7F80830895EFE688
:10447000F0E0908182E08927808308951F920F9257
:104480000FB60F9211242F933F934F935F936F9327
:104490007F938F939F93AF93BF93EF93FF938091FD
:1044A000EB019091EC0101969093EC018093EB016C
:1044B000811103C082E00E94E308E091EC01E695DF
:1044C000E695F0E0EC54FB4FE4918091EB018E1304
:1044D00003C080E00E94E308FF91EF91BF91AF918C
:1044E0009F918F917F916F915F914F913F912F910C
:1044F0000F900FBE0F901F90189504D06894B111C3
:104500008DC0089570D088F09F5790F0B92F9927EB
:10451000B751A0F0D1F0660F771F881F991F1AF0CE
:10452000BA95C9F712C0B13081F077D0B1E00895E3
:1045300074C0672F782F8827B85F39F0B93FCCF364
:10454000869577956795B395D9F73EF490958095C4
:10455000709561957F4F8F4F9F4F0895E89409C0E4
:1045600097FB3EF490958095709561957F4F8F4FA6
:104570009F4F9923A9F0F92F96E9BB279395F695BC
:10458000879577956795B795F111F8CFFAF4BB0F3A
:1045900011F460FF1BC06F5F7F4F8F4F9F4F16C09E
:1045A000882311F096E911C0772321F09EE8872F28
:1045B000762F05C0662371F096E8862F70E060E0E4
:1045C0002AF09A95660F771F881FDAF7880F96955D
:1045D000879597F9089557FD9058440F551F59F046
:1045E0005F3F71F04795880F97FB991F61F09F3FE0
:1045F00079F087950895121613061406551FF2CF09
:104600004695F1DF08C0161617061806991FF1CF58
:1046100086957105610508940895E894BB2766277F
:104620007727CB0197F908950BD078C069D028F08F
:104630006ED018F0952309F05AC05FC01124EECF58
:10464000CADFA0F3959FD1F3950F50E0551F629FED
:10465000F001729FBB27F00DB11D639FAA27F00DDB
:10466000B11DAA1F649F6627B00DA11D661F829F02
:104670002227B00DA11D621F739FB00DA11D621FE7
:10468000839FA00D611D221F749F3327A00D611D04
:10469000231F849F600D211D822F762F6A2F1124E6
:1046A0009F5750408AF0E1F088234AF0EE0FFF1F39
:1046B000BB1F661F771F881F91505040A9F79E3F70
:1046C000510570F014C0AACF5F3FECF3983EDCF3C5
:1046D000869577956795B795F795E7959F5FC1F7AD
:1046E000FE2B880F911D9695879597F9089597F958
:1046F0009F6780E870E060E008959FEF80EC089588
:1047000000240A94161617061806090608950024B0
:104710000A9412161306140605060895092E03942A
:10472000000C11F4882352F0BB0F40F4BF2B11F49E
:1047300060FF04C06F5F7F4F8F4F9F4F089597FBBF
:10474000072E16F4009407D077FD09D00E94B923F4
:1047500007FC05D03EF4909581959F4F0895709584
:1047600061957F4F0895EE0FFF1F0590F491E02DA6
:104770000994AA1BBB1B51E107C0AA1FBB1FA617A8
:10478000B70710F0A61BB70B881F991F5A95A9F7FA
:1047900080959095BC01CD010895F999FECF92BD09
:1047A00081BDF89A992780B50895A8E1B0E042E06C
:1047B00050E00C94F523262FF999FECF92BD81BDD0
:1047C000F89A019700B4021639F01FBA20BD0FB64F
:1047D000F894FA9AF99A0FBE08950196272F0E942D
:1047E000DC230C94DB23DC01CB01FC01F999FECF27
:1047F00006C0F2BDE1BDF89A319600B40D92415069
:0A4800005040B8F70895F894FFCF78
:10480A000220E508730950091C09E8080101C701DB
:10481A0028080A03140A3F4D363975042804F2039E
:10482A00B9034C0365037E039703010203040506DB
:04483A000708090062
:00000001FF
